:1000000018308A0000280000FF00030E8301A100C1
:100010000A08A0008A010408A2007708A300780853
:10002000A4007908A5007A08A6007B08A70083131E
:1000300083128C308400801E1F288C1A39288B1E56
:1000400023280B193628220884002308F7002408E7
:10005000F8002508F9002608FA002708FB00200808
:100060008A00210E8300FF0E7F0E09008A110A12FA
:10007000CB2A8A110A12D52A0A108A100A1182077D
:1000800028340C34013406340A108A100A1182070D
:100090000A3400340E3411341F3411341134003456
:1000A000043400340E3411341F341134113400344C
:1000B000043400340E3401340F3411340F3400345E
:1000C00004340E3415340434043404340434003459
:1000D000043404340434043415340E340434003449
:1000E0000034003400340034003400340034003470
:1000F0000034003400340034003400340034003460
:10010000003400340034003400340034003400344F
:100110000A108A100A118F3E03188A0A820041349D
:1001200001342F344234013406344334013447342B
:100130004434013430344534013409344634013414
:10014000423447340234323448340234343449348B
:10015000023436344A34023438344D34E234003414
:100160004E34E23402344F34E23404345034E23456
:1001700006345134E23408345234E2340A3453340D
:10018000E2340C345434E2340E34583401344E34F6
:10019000593401344F345A34013450344B34E1343F
:1001A00010344C34013453345534E2342034313477
:1001B000E13415343234E13416343334E234173454
:1001C0003434E13419343534E234223436340234F0
:1001D00051343734E2341A343834E2341C3439348C
:1001E000E2341E346134023444346234E134253460
:1001F0006334E13424346434E23426346534013425
:1002000007346634013449346734E13428346834BF
:10021000E23429346934E2342B346A3402346234EF
:100220000A148A100A1182070034003400340034A2
:1002300000340034013400341C34E234003400341F
:10024000443404343C3400342834F1340034003471
:1002500001340034013400341534E1340A340034FC
:1002600063340034013400341634E1340134003492
:100270005A3400340134003416340234013400346A
:1002800001340034013400340A148A100A11820740
:100290000C344534723472346F3472343A3420344E
:1002A000483461347434633468342F340A344F343E
:1002B000763465347234203468346534613474348F
:1002C0006534643400340A148A100A1182070C342D
:1002D000543469346D346534723400340A148A102D
:1002E0000A1182070C344534723472346F3472341C
:1002F0003A3420344F347534743420346F346634D7
:100300000A34503465346C346C346534743473346A
:1003100000340A148A100A1182070C3445347234EE
:1003200072346F3472343A3420344E346F342034A3
:1003300066346C3461346D3465340A346434653445
:1003400074346534633474346534643400340A14AA
:100350008A100A1182070C344534723472346F34B7
:1003600072343A34203448346934673468342F3472
:100370006E34743465346D34703465347234613481
:10038000743475347234653400340A148A100A11D6
:1003900082070C344534723472346F3472343A3418
:1003A000203453346D346F346B34653400340A14A4
:1003B0008A100A1182070C344534723472346F3457
:1003C00072343A342034463465346534643420342D
:1003D000693473340A346134743420346D346934CC
:1003E0006E342034763461346C34753465340034C2
:1003F0000000000000000A108A140A11023E0318CF
:100400008A0A82000C344534723472346F34723488
:100410003A34203455346E346B346E346F34773460
:100420006E340A346534723472346F3472342E345C
:1004300000340A108A140A1182070C344F347034C5
:100440002E34743469346D346534203425346C347E
:1004500075343A34253430343234753420340A3427
:1004600046346534653464342034253464342034AF
:100470002534253420342534633400340A108A149A
:100480000A11820753346134763469346E34673428
:100490002034763461346C347534653400340A1099
:1004A0008A140A1182070C34543469346D3465346B
:1004B00072342034763461346C34753465340034ED
:1004C0000A108A140A11820768346F347534723442
:1004D0007334203400340A108A140A1182070C3451
:1004E000543469346D3465347234203428343134F2
:1004F0003D34533474346F347034293400340A106A
:100500008A140A1182070C344D3461347834203453
:10051000663465346534643400340A108A140A1170
:1005200082070C344D3469346E34203466346534BB
:100530006534643400340A108A140A1182070C34BA
:10054000543465346D3470346534723461347434C9
:100550007534723465340A3425346C346434203490
:1005600025346334433400340A108A140A11820794
:10057000503465346C34323431345F34563465343D
:1005800072345F3432342E34303436340A344534E5
:100590006E3467340034B10BD02A3C140130B10002
:1005A000BD170B118A110A12232818088316DF00C1
:1005B0005F080339003A0319EE2A83121A088316DA
:1005C000DF0083121A088316DF0083121A088316CD
:1005D000DF00831218121816052B831610308312B1
:1005E0006507F800640878020F39F6007608F8000D
:1005F00078080E3C031C052B6630650784001A083A
:100600008000013065070F39E5008C128A110A124B
:100610002328D6308400000803191D2B0130F80070
:10062000F701F70B112BF80B102B4A30F700F70BE3
:10063000172B00000000800B0E2B003483165D0E7C
:10064000F039F7000F3083120805770488000000A6
:10065000081400000000081000348810F0308316E1
:100660008800831208150000081400000808080E0E
:100670000F398316DD0083120810000008140000F3
:100680000808080E0F398316DC00831208100030AA
:10069000831688005D0EF700F030F70577085C04DC
:1006A000F8007808DC00DC1F572B83122E2B5A1819
:1006B0005C2B8312881083165A1C612B83128814BA
:1006C00083160000831208110000081083165B0EC9
:1006D000DC000F30DC055C08DD0083121E2383166E
:1006E0005B080F39DC00DD0083121E23003400306C
:1006F0008316880083128810081108100F308316A3
:10070000D6008312092301308316C3004308033C3B
:10071000031C962B0330DD0083121E230530831645
:10072000D600831209238316C30A862B0230DD000C
:1007300083121E238316C3014308033C031CAD2B05
:10074000430883123C208316C400DA014408DB000E
:1007500083122D238316C30A9C2B0530D6008312E7
:1007600009238316C30143083F3C031CCE2B4030B2
:100770004307C400DA014408DB0083122D238316EB
:100780004308831244208316C4000130DA00440871
:10079000DB0083122D238316C30AB32B83128A1521
:1007A0000A168D2883165508831203178D008316A9
:1007B0008C130C1483120C080313A9002908F800E9
:1007C000003483165308831203178D008316031316
:1007D0005408831203178C0083168C130C15831294
:1007E00003130B138B138B1BF22B5530831603173C
:1007F0008D00AA308D008C14C030831203138B043B
:10080000831603170C11831203130D1A0A2C831677
:100810000317032C0D12003483164E08D3004F0823
:10082000D4008312E123013083164E07D100D0306B
:1008300084000008D2005108D3005208D40083126B
:10084000E123003483165008D5008312D223831687
:10085000D2017808D100D230D30001305007D40043
:10086000D5008312D22383165308840078088000B1
:100870005108F8005208F900831200343D1F9F2CE4
:100880003D130330D5009330D4004E08053C0318C7
:100890009F2C4E08073C031C9F2C60086104031921
:1008A0005A2C60080319E103E00B5A2CE108031DE0
:1008B0005A2CD7141A308316D000831222247908B8
:1008C0008316C6007808C500013045078312DE0094
:1008D000831646088312DF000318DF0A1A308316D6
:1008E000CE0083125F088316D00083125E08831641
:1008F000CF0083120C241C308316D00083122224D4
:1009000079088316C4007808C30043084404031917
:100910009D2C440883125F02031C9B2C031D982C02
:100920005E0883164302031C972C83129B2C8312B0
:10093000C9148430C6009F2C83168312C91000345A
:10094000BD1DA62C3D1DA62C2F14A72C2F10E83062
:1009500083168900831209148316890083120910F3
:100960008316890083120914300893008316141823
:10097000BB2C8312B62C83121308C700E8308316F1
:100980008900831209102F08930083161418CA2CAB
:100990008312C52CE83089008312891483168900DC
:1009A000831289100608F038BF0040083F0203197F
:1009B000DE2C40083F06C1063F08C0000034AF11DE
:1009C000B010BD110E308316D00083122224790896
:1009D000B9007808B8000230B500AE30B400B301F9
:1009E000B201903083168700831207150930CE00BC
:1009F000D30100348316560858068039DA00D61F12
:100A0000062DD509D609D50A0319D60AD81F0D2DEA
:100A1000D709D809D70A0319D80AF801F901F7014B
:100A2000FA015808031D172D57080319312D1030EE
:100A3000D9000310D50DD60DF70DFA0D58087A021E
:100A4000031D242D57087702031C2D2D5708F7028C
:100A5000031CFA035808FA020314F80DF90DD90B18
:100A6000192D0000DA1F392DF809F909F80A0319C0
:100A7000F90A8312003410308316D800F701FA0106
:100A8000D50CD40C031C4A2D5608F7070318FA0A94
:100A90005708FA07FA0CF70CF90CF80CD80B402D94
:100AA00083120034F801F901F701FA0183165608A0
:100AB000031D5D2D55080319772D1030D700031045
:100AC000D30DD40DF70DFA0D56087A02031D6A2DC9
:100AD00055087702031C732D5508F702031CFA030F
:100AE0005608FA020314F80DF90DD70B5F2D00001C
:100AF0008312003420308316D00083122224790818
:100B00008316C9007808C8001530D5008312D22397
:100B100078088316CA001630D5008312D2237808CD
:100B20008316CB002430D5008312D2237808831695
:100B3000CC002530D5008312D22378088316CD004F
:100B40002630D0008312222479088316CF0078083B
:100B5000CE0032304802F7004908FA000030031C8A
:100B60000130FA027708F8007A0883124502031C64
:100B7000C72E031DBF2D440878020318C72E440852
:100B800083164802F7004908FA0083124508031C3F
:100B9000450FFA0277088316C6007A08C70047088F
:100BA000FA004608C71FDD2D4608003CF700FA0191
:100BB0004708031C470FFA027708D0007A08D100D3
:100BC000D11BE92DD108031DAD2E5008FE3C031C9E
:100BD000AD2E4708FA004608C71FF72D4608003C0F
:100BE000F700FA014708031C470FFA027708D00004
:100BF0007A08D100D11B032ED108031D2F2E5008D7
:100C0000273C031C2F2E46088312E2070318E30A31
:100C1000831647088312E307E31B1D2E63082D3C50
:100C200003181D2EFF3A031D192E6208E03C03181D
:100C30001D2E2E30E300E030E200E31F2D2E63086E
:100C4000D13C031C2D2E031D292E62081F3C031CC2
:100C50002D2ED130E3002030E200322E8316831295
:100C6000E301E20163088316D6008312620883164B
:100C7000D5004F08D8004E08D7008312FA24780810
:100C80008316C6070318C70A7908C707FA014C0874
:100C9000D0007A08D1004708D5004608D400510892
:100CA000D7004C08D60083123B2579088316D20062
:100CB0007808D100FA014D08D3007A08D400520810
:100CC000D6005108D5005408D8004D08D70083122B
:100CD000FA2479088316C7007808C6004608323C13
:100CE000C6004708031C470F772E0030782E003CC3
:100CF000C700FA014A08F800FA1F812EC71F8D2E7F
:100D0000832EC71B932E7A084702031C932E031DC4
:100D10008D2E460878020318932EFA014A08C60061
:100D20007A08C700AC2EFA014B08F800C71F9B2EAB
:100D3000FA1FA72E9D2EFA1BAC2E47087A02031C21
:100D4000AC2E031DA72E780846020318AC2EFA011C
:100D50004B08C6007A08C700C52EC71BBC2EC708A3
:100D6000031DB62E4608003C0318BC2EFA014B08A2
:100D7000C6007A08C700C12EFA014A08C6007A08E0
:100D8000C7008312E301E2018316D12E8312FA0118
:100D900083164B08C6007A08C7008312E301E201FC
:100DA000831646088312D30022308316D0008312A4
:100DB000222479088316C5007808C40083123D1CDC
:100DC0000B2F19308316D5008312D2238316D1013D
:100DD0007808D000FA01831253088316D2007A08EB
:100DE000D3005108D5005008D4005308D70052084A
:100DF000D60083123B2579088316D2007808D100EB
:100E00005208D4005108D300D6016430D5008312B3
:100E100052257808D300FA0153088316D0007A08C7
:100E2000D1004508D5004408D4005108D700500827
:100E3000D60083123B2579088316D2007808D100AA
:100E40005208D4005108D300D6016430D500831273
:100E500052257908D2007808D1000034831655084D
:100E6000F80154020318372F5408F700432FF701F5
:100E70000830D600D40DF70D550877020318F70097
:100E8000F80DD60B3A2F831200348316570B492FD7
:100E90004C2F4030D8004D2FD80101305602D807D2
:100EA00058088038D900DA015908DB0083122D2355
:100EB0000034831655080C3A83120319782F063A2A
:100EC0000319842F023A03198C2FEC3A0319932F3C
:100ED000013A03199B2F133A0319A32F323A03192E
:100EE000AB2F013A0319B22F133A0319B92FC12FAF
:100EF0008316DA010130DB0083122D2302308316C2
:100F0000D60083120923C92F01308316D600023080
:100F1000D70083124527C92F8316DA011030DB0072
:100F200083122D23C92F01308316DA00E130DB0054
:100F300083122D23C92F01308316DA000230DB0023
:100F400083122D23C92F01308316DA00EF30DB0026
:100F500083122D23C92F01308316DA00DB0183129F
:100F60002D23C92F01308316DA00DB0083122D23D5
:100F7000C92F01308316DA00EF30DB0083122D23F6
:100F8000C92F01308316DA005508DB0083122D23A8
:100F9000C92F0034F701F80183164C0803104D18CF
:100FA000F707F70CF80CCD18F707F70CF80C4D19EC
:100FB000F707F70CF80CCD19F707F70CF80C4D1ADA
:100FC000F707F70CF80CCD1AF707F70CF80C4D1BC8
:100FD000F707F70CF80CCD1BF707F70CF80C83128A
:100FE00000340C1EF12F83164C0883129900003434
:0C0FF00083164408CC008312F127003463
:1010000004088316D4004E0EF038D000D007E23E1C
:10101000D100323ED3004E080F39D107D107D30794
:10102000E93ED200D207D2074D0E0F39D207D307BF
:10103000D20DD30DD309D30D4D080F39D307D00DE1
:101040000730CF000A30D307D203031C2328D2076E
:10105000D103031C2728D107D003031C2B28D0075A
:10106000CF03031C2F28CF308400073054055413BE
:101070008407D3300402031954170008F700031D36
:101080004928541B4928541A5928D4194928203072
:101090004C28D41554123030F707CE010408CD0087
:1010A0007708D5008A11831259278A1583164D08AF
:1010B0008400840A541F392883128A150A12352C99
:1010C000780883164D08D4006430D5008A11831245
:1010D0002E278A1577088316CD0078083030031D37
:1010E0007828CE1C8328CE1983284E1A20307B28DE
:1010F000CE114E124E14F8077808D5008A118312CB
:1011000059278A1583164D08D4000A30D5008A1154
:1011100083122E278A1577088316CD007808303081
:10112000031D9828CE19A0284E1CA0284E1A203046
:10113000F8077808D5008A11831259278A15831673
:101140003030CD074D08D5008A11831259278A15F2
:101150008A150A12432C203083164F1E3030D000DF
:101160004E08F700CE1FBB28F709F70A7708CE0014
:101170002D30D000CF174E08D4006430D5008A112E
:1011800083122E278A1577088316CE003030780711
:10119000D1004E08D4000A30D5008A1183122E27C0
:1011A0008A15303077078316D30030307807D200A5
:1011B0005008F700CF1DDE28CF1F4F114F1AEB2824
:1011C000CF1F06294F1906297708D100CF18062905
:1011D0007708D200062930305102031D062977080E
:1011E000D1002030D000CF1DF9284F11CF14CF1FD0
:1011F000CF1030305202031D06297708D20020306C
:10120000D100CF1DF928CF10CF1F4F104F1D0F2930
:101210005008D5008A11831259278A158316CF1CCE
:1012200018295108D5008A11831259278A15831667
:101230004F1C21295208D5008A11831259278A157B
:1012400083165308D5008A11831259278A158A15E7
:101250000A12602C04088316D100CB1F3729D1173E
:10126000511ED10ACA09CB09CA0A0319CB0A4B0E6F
:10127000F038CD00CD07E23ECE00323ED0004B0824
:101280000F39CE07CE07D007E93ECF00CF07CF07F3
:101290004A0E0F39CF07D007CF0DD00DD009D00D92
:1012A0004A080F39D007CD0D0730CC000A30D007DF
:1012B000CF03031C5729CF07CE03031C5B29CE079E
:1012C000CD03031C5F29CD07CC03031C6329CC305D
:1012D000840007305105511384035105031D7729FC
:1012E000511A840A511A77292030F700942984076B
:1012F000D0300402031951170008F700031D882994
:10130000511B8829511AA029D119882920309329E5
:10131000D11F90292D30F70084035113D113942944
:10132000D11551123030F707CB010408CA007708F5
:10133000D5008A11831259278A1583164A0884001A
:10134000840A511F782983120034831644080B3C09
:10135000031DB5291A30CE00D001CF018A118312A6
:101360000C248A15DF01DE0183164408083C031DA6
:10137000C52A0130831248078316CA00D4000630FC
:10138000D5008A1183122E278A1577088316C60086
:10139000460DF700F70DF70DF830F7057708013E19
:1013A0008A11831210218A15F8008316C700470896
:1013B000DF3C0318C52A460DF700F70DF70DF8308E
:1013C000F7057708043ECA004A0A8A1183121021E1
:1013D0008A15FA0083164A088A11831210218A1589
:1013E000DA007A08DB008316460DF700F70DF70DDB
:1013F000F830F7057708023ECA004A0A8A118312BC
:1014000010218A15FA0083164A088A1183121021C6
:101410008A15DC007A08DD008316460DF700F70D0B
:10142000F70DF830F70577088A11831210218A1515
:10143000F8008316C8004708E13C031D4B2A480802
:10144000D5008A118312D2238A1578088316C90021
:10145000460DF700F70DF70DF830F7057708063E53
:10146000CB004B0A8A11831210218A15FA008316C9
:101470004B088A11831210218A158316CC00490863
:10148000D4004C08D5008A1183122E278A15D90161
:101490007808D80083164708E23C031D842A4808D0
:1014A000D0008A11831222248A1579088316CA0073
:1014B0007808C900460DF700F70DF70DF830F7056D
:1014C0007708063ECC004C0A8A11831210218A1537
:1014D000FA0083164C088A11831210218A1583168C
:1014E000CD007A08CE004A08D4004908D3004E083F
:1014F000D6004D08D5008A11831252258A15790825
:10150000D9007808D80083164708EF3C0318A32AAF
:101510004808D5008A118312D2238A1578088316C9
:10152000C90047080739F8004908F700F808031907
:101530009D2A0310F70CF80B992A770801398312BA
:10154000D800D901831683125B085902031CB22A02
:10155000031DAE2A58085A020318B22A5B08D900A4
:101560005A08D80059085D02031CC02A031DBC2A72
:101570005C0858020318C02A5D08D9005C08D8002E
:101580005714BB019830BA00831644080A3C031D67
:10159000F72A8312C908031DCF2A8316F72A0130C0
:1015A000F7004A08F8000319D92A0310F70DF80BC1
:1015B000D52A7708FF3AC905BB010230BA004A08AC
:1015C000FB3E0318F62A053EA42EF62A1A3083168F
:1015D000CE00D001CF018A1183120C248A15DF01BD
:1015E000DE01F62AC201F62A3D12F62A83164408C5
:1015F000453C031D812C831257104E080B3C031DE4
:101600000B2B49084B05003A031D0B2BCE01BC13D5
:101610003C13D001CF01C9080319E62B8316C5017D
:101620004508073C031CE42B8312CA0A0730CA058D
:101630004908F7004A08F8000319222B0310F70C99
:10164000F80B1E2B771CE12B4A08F83E0318DA2B07
:10165000083EAD2E8316C90149088A118312442120
:101660008A158316C90AF700D5008A1183125927F3
:101670008A151A3083164902031D2C2B8312DA2B8C
:101680008316C90149088A11831263218A158316BA
:10169000C90AF700D5008A11831259278A15063026
:1016A00083164902031D422B8312DA2B8316C901CC
:1016B00049088A1183126E218A158316C90AF70018
:1016C000D5008A11831259278A15163083164902CC
:1016D000031D582B8312DA2B8316C90149088A117E
:1016E000831289218A158316C90AF700D5008A1149
:1016F000831259278A15193083164902031D6E2B50
:101700008312DA2B8316C90149088A118312A72193
:101710008A158316C90AF700D5008A118312592742
:101720008A15193083164902031D842B8312DA2B84
:101730008316C90149088A118312C5218A158316A7
:10174000C90AF700D5008A11831259278A150D306E
:1017500083164902031D9A2B8312DA2B8316C901C3
:1017600049088A118312D7218A158316C90AF700FE
:10177000D5008A11831259278A151C308316490215
:10178000031DB02B8312DA2B8316C90149088A1175
:101790008312F8218A158316C90AF700D5008A1129
:1017A000831259278A15163083164902031DC62B4A
:1017B0008312DA2BC801BB012D30BA008316E42B4B
:1017C00083128316C50A102B812C83123F08F93C23
:1017D000031DF52B1A308316CE00D001CF018A11DC
:1017E00083120C248A15DF01DE015F088316D40002
:1017F00083125E088316D300D6013C30D5008A11CF
:10180000831252258A1579088316CA007808C90000
:1018100083125F088316D40083125E088316D300F8
:10182000D6013C30D5008A11831252258A157708DB
:101830008316CB00CC014C088A11831219228A1519
:101840008316CC0AF700D5008A11831259278A150E
:10185000093083164C02031D1B2C103084004A08EB
:10186000CE004908CD00831200283A308316D500F7
:101870008A11831259278A1583164B08CD0001302F
:10188000CE008312602811308316CD004D088A11D6
:10189000831219228A158316CD0AF700D5008A1102
:1018A000831259278A15183083164D02031D462CC2
:1018B000831253088316CE001F30CF008312AB284B
:1018C00020308316D5008A11831259278A152530B6
:1018D0008316D5008A11831259278A152030831662
:1018E000D5008A11831259278A154D088316D50011
:1018F0008A11831259278A15C801BB010F30BA001B
:1019000083164408093C031D7A2D831257188A2C2C
:1019100083167A2D5710480DF700F70DF70DF830A4
:10192000F7057708013E8A1110218A15F800831601
:10193000C7008312480DF700F70DF70DF830F705D3
:1019400077088A1110218A15F8008316C800470805
:10195000E13C031DDA2C8312480DF700F70DF70D5B
:10196000F830F7057708063E8316CA004A0A8A113E
:10197000831210218A15FA0083164A088A118312ED
:1019800010218A158316CB00831258088316CC00C9
:101990004B08CD008A118312CA278A15780883164E
:1019A000CC004808D3004C08D4008A118312E123EC
:1019B0008A1583164708E23C031D192D8312480D32
:1019C000F700F70DF70DF830F7057708063E831698
:1019D000CA004A0A8A11831210218A15FA00831656
:1019E0004A088A11831210218A158316CB007A08BF
:1019F000CC00831259088316D50083125808831629
:101A0000D4004C08D7004B08D6008A1183123B251E
:101A10008A1579088316CD007808CC004808CE00D6
:101A20004D08D0004C08CF008A1183120C248A156F
:101A300083164708EF3C0318562D4808D5008A1135
:101A40008312D2238A1578088316C5008312D8081A
:101A500003193C2D831647080739C9000130F700E8
:101A60004908F8000319382D0310F70DF80B342D31
:101A70007708C5044D2D8312831647080739C9001E
:101A80000130F7004908F80003194A2D0310F70D3B
:101A9000F80B462D7708FF3AC5054808D3004508DE
:101AA000D4008A118312E1238A1583168312C80198
:101AB00001308316D6000230D7008A1183124527E1
:101AC0008A158316C90149088A1183123E228A1594
:101AD0008316C90AF700D5008A11831259278A157F
:101AE0000C3083164902031D632D8312BB010F3096
:101AF000BA00831683124808FA3E0318A12E063E48
:101B0000B92E83164408083A8312031DBB2D831691
:101B1000C90149088A1183124F228A158316C90AFE
:101B2000F700D5008A11831259278A150C308316C5
:101B30004902031D892D0A30D6000230D7008A11D0
:101B4000831245278A158316C90149088A11831211
:101B500060228A158316C90AF700D5008A118312FC
:101B600059278A15063083164902031DA52D013019
:101B70008312C800BB2DA12E83164408083A831295
:101B8000031DDA2D8316C90149088A1183126B22BD
:101B90008A158316C90AF700D5008A1183125927BE
:101BA0008A150F3083164902031DC42D023083129B
:101BB000C800DA2DA12E83164408083A8312031DAB
:101BC000172E8316C90149088A1183127F228A15AC
:101BD0008316C90AF700D5008A11831259278A157E
:101BE000093083164902031DE32D03308312C80018
:101BF0000A308316D6000230D7008A118312452797
:101C00008A1525308316D5008A11831259278A1523
:101C100020308316D5008A11831259278A15203067
:101C20008316D5008A11831259278A15172EA12EE3
:101C300083164408083A8312031D542E8316C901E3
:101C400049088A1183128D228A158316C90AF70062
:101C5000D5008A11831259278A1509308316490243
:101C6000031D202E04308312C8000A308316D600CC
:101C70000230D7008A11831245278A152530831632
:101C8000D5008A11831259278A1520308316D50072
:101C90008A11831259278A1520308316D5008A119C
:101CA000831259278A15542EA12E83164408083A08
:101CB0008312031D932E0530C8008316C9014908FD
:101CC0008A1183129B228A158316C90AF700D50050
:101CD0008A11831259278A150D3083164902031D74
:101CE0005F2E10308400831245088316CB008312C8
:101CF00044088316CA0083122A2120308316D50097
:101D00008A11831259278A15DF308316D5008A116C
:101D1000831259278A1543308316D5008A118312FE
:101D200059278A15932EA12E83164408083A831248
:101D3000031DA02EC8015710BB010230BA00A02E0F
:101D4000A12E8A110A16FA2A0A108A140A15820785
:101D5000E52AE62AF32AF22AF42A0A108A140A1536
:101D600082072A2B402B562B6C2B822B982BAE2BC9
:101D7000C42B0A108A140A158207812DBC2DDB2D75
:101D8000182E552E942E20308316C4008A118312EB
:101D9000F8278A1556308316C4008A118312F82753
:101DA0008A158316C30143088A118312B4228A1547
:101DB0008316C30AF700C4008A118312F8278A1514
:101DC000123083164302031DD32E0D30C4008A1136
:101DD0008312F8278A1500343D153208330403199D
:101DE000F92E32080319B303B20BF92EB308031905
:101DF000BC14340835040319052F34080319B5033E
:101E0000B40B052FB50803193C1536083704031920
:101E1000112F36080319B703B60B112FB708031992
:101E2000BC153808390403191D2F38080319B903E4
:101E3000B80B1D2FB90803193C163A083B040319C7
:101E4000292F3A080319BB03BA0B292FBB08031922
:101E5000BC16540855040319352F54080319D5032B
:101E6000D40B352FD50803193D17D6080319392F80
:101E7000D6038A150A163D2A6630640784000008D6
:101E8000FC0083168C120130831264070F39E400C2
:101E900083168C167C08F80083128A150A16442AC9
:101EA00083164508393C031C5A2F30304502F80090
:101EB0005F2F5F2F4508DF39C93EF8005F2F83127F
:101EC00000348316CB1B782F0F30F7004A0EF7052E
:101ED0000A30770203186F2F3030F707712F4B0845
:101EE000F7077708CC008A118312F1278A15831629
:101EF0000F30CA050A304A020318802F3030822F73
:101F0000CB134B08CA074A08CC008A118312F12769
:101F10008A1500348316C908031D982F4608AB00A4
:101F20004708AC004808AD008312D716C42F8316AB
:101F3000C9080319C52F8312D71AA02F8316C52FDE
:101F400020308316CC008A118312F1278A1583165C
:101F50002B08CC008A118312F1278A1583162C08CE
:101F6000CA003730CB008312612783162D08CA00C0
:101F70003730CB00831261270D308316CC008A11D5
:0E1F80008312F1278A15D712831683120034BC
:102000008316430F19288312B301B201B501B4013D
:10201000B701B601B901B801BC103C11BC113C12AA
:10202000BC133C13BD10CE01D001CF01CC01162B47
:10203000831683124C08003A03192228013A031927
:1020400031284728491483164308853C031D2F284F
:1020500001308312CC004910CE01D30183168312C4
:10206000472883164308053C031D45288312CC01ED
:102070000B30CE00AF01B001903083168700831281
:102080000711BD114914D301831683124728500844
:10209000003A03194F28013A03195A286228831677
:1020A0004308813C031D582801308312D000831659
:1020B000831262288316430B60288312D001831693
:1020C000831262284F08003A03196A28013A03195B
:1020D00075287F2883164308023C031D73280130AE
:1020E0008312CF00831683127F2883164308823C15
:1020F000031D7D288312CF01831683127F284E088B
:10210000F13E0318F32A0F3E172B4B084905003AFE
:1021100003198D280B30CE00F32A4F0BB0284C0B3F
:10212000B028BD1EB0288316D0010A1283122224C3
:102130000A167908B3007808B200AF15AF16AF14CD
:10214000AF172F152F162B308316D0000A128312CB
:1021500022240A167908E1007808E0000130CE0058
:10216000F32A83164308413A83120319BB28C33A62
:102170000319D228D728AF11AF12B01490308316AC
:10218000870083120715BD150A308316D0000A1286
:10219000831222240A167908B5007808B4000230A8
:1021A000CE00D7280A12DF240A16AF12D728F32A46
:1021B000500BE8281E308316D0000A128312222406
:1021C0000A167908B5007808B4000330CE00F32A67
:1021D00083164308423A83120319F228C03A0319BE
:1021E0000A290F29BD11B010AF1190308316870056
:1021F00083120711AF120C308316D0000A1283121B
:1022000022240A167908B3007808B200C20A0830FE
:10221000CE000F290A12DF240A16AF120F29F32A63
:1022200083164308423A831203191A29C03A031944
:102230003229362990308316870083120715B01093
:10224000BD1104308316D0000A12831222240A160C
:102250007908B5007808B40004308316AA00831208
:10226000CE0036290A12DF240A163629F32A8316ED
:102270004308423A831203194129C03A03196029DD
:102280006529AF168316AA0B53290630D0000A120F
:10229000831222240A167908B5007808B4000530A4
:1022A000CE00652983160230D0000A128312222440
:1022B0000A167908B5007808B4000C30CE006529FC
:1022C0000A12DF240A16AF126529F32A831643087F
:1022D000423A831203197029C03A03197F298429CD
:1022E000AF1208308316D0000A12831222240A1675
:1022F0007908B5007808B4000430CE0084290A12A9
:10230000DF240A16AF128429F32A83164308423ABF
:10231000831203198F29C03A031999299D29AF11F6
:10232000AF12B301E430B200B014BD150E30CE00D0
:102330009D290A12DF240A169D29F32A83164308D1
:10234000423A83120319B129013A0319B429C73A51
:102350000319D529063A0319D629833A0319DA292C
:10236000F1293D10C201F129AF110A127A250A168E
:1023700022308316D0000A12831222240A1679080A
:102380008316C5007808C4008312510883164402DE
:102390008312B600831645088312B7005208031C47
:1023A000520FB7020730CE00F129F1290A12DF24BB
:1023B0000A16F129D301AF119030831687008312DA
:1023C0000711AF120C308316D0000A128312222498
:1023D0000A167908B3007808B200C20A0830CE00A5
:1023E000F129F32A83164308423A83120319052A76
:1023F000013A0319082AC73A0319102A063A0319A1
:10240000112A833A0319152A2C2A3D10C2012C2ABD
:10241000AF155208B7005108B6000630CE002C2A7E
:102420002C2A0A12DF240A162C2AD301AF1190306D
:102430008316870083120711AF120C308316D00069
:102440000A12831222240A167908B3007808B2000F
:10245000C20A0830CE002C2AF32A83164308413AD8
:102460008312031D522A4F0B4A2A10308316D500BF
:102470000A128312D2230A167808420203184A2A43
:10248000BD1E4A2AAF16AF15B5019830B4000A3008
:10249000CE00512AC915AF10AF132F112F120B30D8
:1024A000CE00522AF32A83164308413A83120319B5
:1024B000602A033A0319662A063A0319702A812A08
:1024C00090308316870083120715812A9030831677
:1024D0008700831207110A30B300BA30B200812A94
:1024E000AF1290308316870083120711AF10AF131D
:1024F0002F112F122F17B5015B30B4000D30CE0015
:10250000812AF32A83164308423A8312031D9F2A25
:102510000A308316D0000A12831222240A16790880
:10252000B5007808B400AF11AF12B014BD159030EB
:1025300083168700831207150230CE009F2AF32AE4
:10254000831643080A3A8312031DA72AA72AF32AEF
:1025500083164308423A8312031DB12A2F13CE017A
:10256000B12AF32A83164308413A83120319BC2A7D
:10257000C33A0319EE2AF22AB010BD11500BD82A23
:10258000AF15AF163D1417308316D0000A12831210
:1025900022240A167908B5007808B4000A127A25B0
:1025A0000A165208B7005108B6000630CE00ED2AD0
:1025B000AF1190308316870083120711AF120C30D1
:1025C0008316D0000A12831222240A167908B30057
:1025D0007808B200C20A0830CE00F22A0A12DF24BC
:1025E0000A16F22AF32A83164308C4000A128A152F
:1025F0008312A5290A168A11C90803190B2B9030DA
:1026000083168700831287143014E83083168900FC
:1026100083120915162B90308316870083128710BA
:102620003010E830831689008312091100340A142F
:102630008A140A1182078528B128D8281029372939
:1026400085299E29F2292D2A532A822AA02A662921
:10265000A82AB22A831606168312061E4C2B571977
:102660004A2B57158316861600308312861A0130BE
:10267000003A031D492B59085B02031C482B031D1C
:10268000452B5A0858020318482BD80A0319D90AAF
:10269000492B4B2B682B682B571D672B5711831623
:1026A000861600308312861A0130013C0319662B0E
:1026B0005D085902031C662B031D622B58085C023F
:1026C0000318662B58080319D903D803682B682B05
:1026D0008316200883125802031D742B83162108C9
:1026E000831259020319792B571C792BBB0198309F
:1026F000BA0059088316A100831258088316A00057
:1027000083128A150A16FE2B571EEC2B83162808F7
:102710000F3C0318D12BA801270CC600260CC500BE
:10272000C60CC50CC60CC50CC60CC50CC60CC50C1D
:102730000730C60545088312C400023083164607D9
:102740008312C5004508023C031CAE2B031DAC2BB5
:1027500044081B3C031CAE2BBD16AF2BBD124E080C
:10276000093C0319CD2B4E080D3C0319CD2BCE0887
:102770000319CD2B29308316D0000A12831222248C
:102780000A167908FA007A084502031CCD2B031DAE
:10279000CC2B44087802031C49168316A701A60116
:1027A000E32B83121F151F19D32B1E08FA00831663
:1027B0001E08C3007A08C4004308A6070318A70A26
:1027C0004408A707A80A0830F80083121F08C73971
:1027D00078049F005712FA2B1F151F19ED2B831633
:1027E0001E088312C3000030F8001F08C7397804A0
:1027F0009F0057168A150A16112C47088316A50044
:10280000A5092830D5000A128312D2230A167808A7
:10281000CB00BC1C0F2CBC104130F8002A2D3C1DF5
:10282000152C3C114230F8002A2DBC1D1B2CBC116C
:102830004330F8002A2D3C1E212C3C124430F80075
:102840002A2DBC1E272CBC124530F8002A2DBD1C99
:10285000342C8316A51B322C8312BD100530F800D2
:102860002A2D83163D2C83128316A51F3D2C83121F
:10287000BD148530F8002A2D83168312471C432C83
:102880004230CD00452C2030CD00BC1F572C4708CE
:102890000139003A031D542CD608031D532CBC13D8
:1028A0000130F8002A2D562CE430D6005F2C471C4E
:1028B0005F2CE430D600BC178130F8002A2DD71CDD
:1028C000662CD7103C138230F8002A2D3C1F752C43
:1028D0008316A51C6D2CA519732C83123C13823012
:1028E000F8002A2D8316822C83128316A51C822CB5
:1028F000251D822CA51D822C83123C170230F80066
:102900002A2D83168312C6080319902C46088316B5
:10291000A5008312C60183162508F80083122A2D0C
:102920008316251EA32C831249080439003A031D7F
:10293000A02C4B1DA02C3C1349158230F8002A2DE9
:102940004915A52C8316831249118316A51EB72C91
:10295000831249082039003A031DB52CCB1EB52C33
:102960003C13C9168230F8002A2DC916831683122B
:102970003D1AC32C491EC32C4B1EC32C3C133D16C1
:102980008230F8002A2D41083F05003A0319F52C42
:102990008316A3012308073C031CF42C0130A40078
:1029A0002308F8000319D82C0310A40DF80BD42C1D
:1029B000831241083F0583162405003A0319F22CBF
:1029C0002408FF3A8312C1058316220EF700F03067
:1029D000F7057708803E2307013E073EF800831283
:1029E0002A2D8316A30ACA2C83123F08FF3A4105F9
:1029F000003A0319282D8316A3012308073C031C62
:102A0000272D0130A4002308F80003190B2D031013
:102A1000A40DF80B072D83123F08FF3A41058316DA
:102A20002405003A0319252D2408FF3A8312C10515
:102A30008316220EF700F030F70577082307013ED2
:102A4000073EF80083122A2D8316A30AFD2C831259
:0A2A50000030F8008A150A16162C53
:103000001F3083055730F700203084008001840A88
:10301000F70B0628F801F901FA01FB01FC01FD019B
:10302000FE015030F700A03084008001840AF70BC5
:103030001528A00184011F30830583161F149F14D7
:103040001F159F110C309900263098009030831284
:103050009800A801A901AA010130AB00AC01AD01A3
:10306000AE01F601FC015711D7118316A001A10191
:10307000A201A301A401A501831257128316A60180
:10308000A701A801A901AA01AB01AC01AD018312FE
:10309000D7128316B2018312D30114308316D600DF
:1030A0000A128A11831209230A168A153D10C601D5
:1030B0000730F700F71D6428073081018130840054
:1030C0000008C0390F388000640081308400000897
:1030D000C0397704800083161F149F101F159F119D
:1030E00083121F179F1783169F1783121F149412A2
:1030F0009030831687008700870030308312940059
:103100004030831694000030F80083121F08C7393E
:1031100078049F000A128A11772B0A168A1501304B
:103120008316D5000A128A118312D2230A168A1531
:10313000780FC9298316CE010230D0001630CF0097
:103140000A128A1183120C240A168A1564000230AE
:103150008316CE00D0011E30CF000A128A118312CE
:103160000C240A168A15640004308316CE00D001A0
:10317000E430CF000A128A1183120C240A168A1531
:10318000640006308316CE000130D0003130CF000D
:103190000A128A1183120C240A168A1564000A3056
:1031A0008316CE000730D0002730CF000A128A11D4
:1031B00083120C240A168A15640008308316CE0088
:1031C0000130D0007D30CF000A128A1183120C2406
:1031D0000A168A1564001E308316CE000230D00015
:1031E0001630CF000A128A1183120C240A168A158F
:1031F00064000C308316CE000130D0003130CF0097
:103200000A128A1183120C240A168A1564000E30E1
:103210008316CE003530D000A430CF000A128A11B8
:1032200083120C240A168A15640010308316D3000A
:103230000430D4000A128A118312E1230A168A1577
:10324000640015308316D3005A30D4000A128A1154
:103250008312E1230A168A15640016308316D30000
:103260001430D4000A128A118312E1230A168A1537
:10327000640017308316CE000630D0008E30CF00A9
:103280000A128A1183120C240A168A156400193056
:103290008316D3003C30D4000A128A118312E12332
:1032A0000A168A151A308316CE00D001CF010A12F1
:1032B0008A1183120C240A168A1564001C308316A6
:1032C000CE00D001CF010A128A1183120C240A16F3
:1032D0008A1520308316CE000230D000BC30CF00DB
:1032E0000A128A1183120C240A168A1522308316B8
:1032F000CE00D0015B30CF000A128A1183120C2459
:103300000A168A1525308316D3000830D4000A1215
:103310008A118312E1230A168A1524308316D300FA
:103320000430D4000A128A118312E1230A168A1586
:10333000640026308316CE00D0013230CF000A124E
:103340008A1183120C240A168A1528308316D3009A
:103350003E30D4000A128A118312E1230A168A151C
:1033600029308316CE000330D0005230CF000A122D
:103370008A1183120C240A168A152B308316CE006C
:10338000D001F030CF000A128A1183120C240A16E1
:103390008A15D301FF30BF00C000C101831642105F
:1033A0008312D710C901CA01BD110730BE00033016
:1033B000D5009330D4003D17C9100630CE000A1254
:1033C0008A113E240A168A15CE01C8015710C2017F
:1033D000E401E501AF01B00190308316870083124C
:1033E00007110A128A11A0240A168A15FF308316C3
:1033F000C3008A11831200208A150A12C3260A16F6
:103400008B1683168C16C03083128B048316B3017F
:1034100001308312B1000C308316D5000A128A11D4
:10342000831259270A168A158316C30143080A1204
:103430008A118312B4220A168A158316C30AF7006A
:10344000D5000A128A11831259270A168A151230DA
:1034500083164302031D162A8312BC12BB01983047
:10346000BA003D1290308316870083120710640063
:10347000BD1F3E2ABD130A12EC2E0A16650864020F
:103480000319FA2B0A123C2F0A1678088316B1008A
:103490003108203C031D4F2A0130B200FB2BB2083B
:1034A0000319FB2B31080D3C031DBC2B03303202EA
:1034B000F83E0318BA2B083E8312892C8316BA2BC8
:1034C0008316BA2B83163808C5000A1283125027B8
:1034D0000A16780E8316C400F030C4053908C500FA
:1034E0000A12831250270A16780883164407B80078
:1034F0003A08C5000A12831250270A16780E83165E
:10350000C400F030C4053B08C5000A1283125027DE
:103510000A16780883164407B9003708563C031D7D
:10352000972A0A128312C3260A168316BA2B370863
:10353000573C031DA02A38088312C6008316BA2BF5
:10354000B50135082A3C031CB82B3508CC000330E4
:10355000CD000A128A118312CA270A168A15780822
:103560000A128A1188200A168A15F8008316BC00F0
:1035700037083C02031DB62B3508CC000330CD00C4
:103580000A128A118312CA270A168A15013078078F
:103590000A128A1188200A168A15F8008316BD00BF
:1035A0003508CC000330CD000A128A118312CA27D5
:1035B0000A168A15023078070A128A1188200A161C
:1035C0008A15F8008316BE00BD080319B52B3D0B04
:1035D000052B3608573C031DF52A3208053C031D10
:1035E000F52A3E088400380880003E088400000860
:1035F000C3003708C600C7014308C800C9010A1242
:1036000083128A270A16B42B83163D08023C031D39
:10361000302B3608573C031D1A2B3208073C031D7C
:103620001A2B3E0884003908800001303E078400D0
:103630003808800001303E0784000008C3003E08BF
:1036400084000008C4003708C6004308C7004408C7
:10365000C800C9010A1283128A270A16B42B8316DE
:103660003D08E03C0319B52B3D08E13C031D622BEE
:103670003608573C031D4B2B3208053C031D4B2BD2
:103680003E08D3003808D4000A128A118312E123BD
:103690000A168A1583163E08D5000A128A1183126B
:1036A000D2230A168A1578088316C3003708C60085
:1036B000C7014308C800C9010A1283128A270A16E3
:1036C000B42B83163D08E23C031DAB2B3608573C58
:1036D000031D862B3208073C031D862B01303E0755
:1036E000C300D3003808D4000A128A118312E123E0
:1036F0000A168A1583163E08D3003908D4000A1228
:103700008A118312E1230A168A15831601303E07B7
:10371000C300D5000A128A118312D2230A168A1511
:1037200078088316C4003E08D5000A128A11831255
:10373000D2230A168A1578088316C5003708C600F2
:103740004408C7004508C800C9010A1283128A2725
:103750000A16B42B83163708C600C701C801C90171
:103760000A1283128A270A168316B82BB50AA12AD1
:10377000BA2B8316B201FB2B01303202F73E03183D
:10378000FB2B093E8312952C83163108B6000230BC
:10379000B200FB2B83163108B7000330B200FB2BBD
:1037A00083163108B8000430B200FB2B83163108B1
:1037B000B9000530B200FB2B83163108BA00063081
:1037C000B200FB2B83163108BB000730B200FB2B85
:1037D00083163108BC000830B200FB2B8316310879
:1037E000BD000930B200FB2B83163108BE000A3041
:1037F000B200FB2B83168A1183122A2B8A1583169B
:103800003308FB3E0318812C053E8312A22C3C1C7E
:10381000122C3C100A128A11A0240A168A158A1149
:10382000842B8A158316812C8A11FD2B8A15780822
:103830008316B4003408C3008A11831200208A154D
:103840008316B4080319312C421C312C5730C600A2
:10385000C7013408C800C9010A1283128A270A1650
:103860008316812C0A128A113E240A168A158316A1
:10387000812C571C722C480DF700F70DF70DF8300E
:10388000F7057708013E0A128A1110210A168A15D7
:10389000DF3C0318722C01308316D6000230D700AB
:1038A0000A128A11831245270A168A1510308400DD
:1038B00059088316CB00831258088316CA000A12CF
:1038C00083122A210A1604308316C3002030D50043
:1038D0000A128A11831259270A168A158316C30BF6
:1038E000662C83128316812C8316C601C701C8017A
:1038F0000130C9000A1283128A270A168316812C06
:103900008316B30A3308053C0319B3018312372A1F
:1039100063000A108A100A158207622A5E2A622A48
:10392000B92B622AB92BB92B602A0A108A100A1502
:103930008207C42BCA2BD02BD62BDC2BE22BE82BF7
:10394000EE2BF42B0A108A100A158207072C142C70
:06395000322C392C742C0E
:02400E00723FFF
:00000001FF
